:10000000B201BC28A501A400B3172730A30010300B
:1000100015200330A300E8301520A301643015201B
:10002000A3010A30152024082028A2002508A100D9
:100030002408A0009B202008031DB313B31B080055
:10004000303EA70089100911091183168910091182
:100050000911F030880583122708B2184D283A306C
:10006000A10098307F203330A60062201330A10019
:1000700088307F20622064307E20622064307E20C1
:100080002230A600622028304C200C304C20063054
:100090004C20B21427084D283214A600321C5B28CD
:1000A0000911033C031C602860200730A100D030F8
:1000B0007F20031408003214FE3C0319B7280915E9
:1000C000A60E321C32108914F030880526080F392C
:1000D00088048910A60E3218622832307E2003145C
:1000E0000800A301A200FF30A207031CA307031C02
:1000F000B7280330A100DF307F207328A101E83E3C
:10010000A000A109FC30031C8828A007031885283B
:10011000A0076400A10F852820188E28A01C922813
:100120000000922808000038031DFF3084080319DE
:10013000B728FF3AB728A501A4011030A600210D69
:10014000A40DA50D2208A4022308031C230FA50259
:100150000318B1282208A40723080318230FA507B2
:100160000310A00DA10DA60B9F282008B72883130C
:100170000313831264000800831607309F000F30BA
:1001800085008601831286010130A300F4308A01C4
:100190007220FE308A01212001308A012120203086
:1001A0008A01212020308A01212020308A0121204B
:1001B00049308A01212059308A01212049308A01A1
:1001C000212020308A01212047308A01212055300A
:1001D0008A0121204E308A0121204C308A012120C1
:1001E00045308A01212052308A012120FE308A01C7
:1001F0002120C0308A01212020308A012120203096
:100200008A01212044308A01212054308A01212092
:100210004D308A01212046308A01212020308A0178
:10022000212020308A0121204B308A0121204F30AB
:100230008A0121204E308A01212054308A01212058
:1002400052308A0121204F308A0121204C308A010E
:1002500021200F300505BA0064003A08003C8A11DD
:100260000A1203192929640009303A028A110A1274
:100270000318B3298A110A12752338088604FE3040
:100280008A01212001308A01212020308A01212089
:1002900020308A0121203A088A0102202E308A016A
:1002A00021204B308A01212041308A0121204E300B
:1002B0008A01212041308A0121204C308A012120ED
:1002C00020308A01212041308A0121204B308A01CF
:1002D000212054308A01212049308A0121204630D2
:1002E0008A012120FE308A012120C0308A0121208C
:1002F00020308A01212045308A01212052308A0194
:1003000021204B308A01212041308A0121204E30AA
:100310008A01212020308A01212026308A012120D3
:1003200020308A01212042308A01212045308A0173
:10033000212052308A01212048308A012120413079
:100340008A0121204E308A0121200F300505B90095
:100350003A08840039088A0193208A110A12031D81
:1003600029298A01A52964003A080A3C8A110A123F
:10037000031D122A8601FE308A01212001308A01E4
:10038000212020308A01212020308A012120543070
:100390008A01212055308A0121204D308A012120F7
:1003A00020308A0121204B308A01212041308A01EE
:1003B00021204E308A01212041308A0121204C30F9
:1003C0008A0121204C308A01212041308A012120DC
:1003D00052308A012120FE308A012120C0308A015A
:1003E000212020308A01212020308A012120203044
:1003F0008A01212020308A01212020308A012120F9
:1004000020308A01212050308A01212041308A0188
:10041000212053308A01212049308A012120463091
:100420008A01212064003A080B3C8A110A12031D3C
:10043000702B01308A0171200F300505B90064006E
:1004400039080B3C8A110A12031D282A8A01192A2D
:10045000FE308A01212001308A01212020308A01CA
:10046000212020308A01212048308A01212041307A
:100470008A0121204E308A01212047308A01212023
:1004800049308A01212020308A01212020308A0130
:1004900021204B308A01212041308A0121204E3019
:1004A0008A01212041308A0121204C308A012120FB
:1004B000FE308A012120C0308A01212020308A01AB
:1004C000212020308A01212020308A0121204B3038
:1004D0008A01212041308A01212050308A012120C7
:1004E00041308A01212054308A01212049308A017B
:1004F00021204C308A01212053308A0121204930AB
:100500008A0121204E308A0121200F300505B900D3
:10051000000064003908003C8A110A120319852A78
:100520000F300505BA008A110A127523060838052E
:10053000B90064003908003C8A110A1203190B2B18
:1005400038088606FE308A01212001308A012120E8
:1005500020308A01212020308A0121203A088A0196
:1005600002202E308A0121204B308A012120413087
:100570008A0121204E308A01212041308A01212028
:100580004C308A01212020308A01212050308A01FC
:10059000212041308A01212053308A012120493015
:1005A0008A01212046308A012120FE308A01212043
:1005B000C0308A01212020308A01212045308A0163
:1005C000212052308A0121204B308A0121204130E4
:1005D0008A0121204E308A01212020308A012120E9
:1005E00026308A01212020308A01212042308A01D0
:1005F000212045308A01212052308A0121204830B3
:100600008A01212041308A0121204E308A01212097
:100610008A110A12622BFE308A01212001308A01E0
:10062000212020308A01212020308A012120203001
:100630008A01212020308A01212042308A01212094
:1006400055308A01212020308A01212020308A0162
:10065000212020308A0121204B308A012120413085
:100660008A0121204E308A01212041308A01212037
:100670004C308A012120FE308A012120C0308A01BD
:10068000212002308A01212020308A0121202030BF
:100690008A01212020308A01212020308A01212056
:1006A00020308A01212050308A01212041308A01E6
:1006B000212053308A01212049308A0121204630EF
:1006C0008A0121200F300505B9003A088400390855
:1006D0008A0193208A110A12031D29298A01622B9B
:1006E00004308A0171208A0129293A08083C8A11BC
:1006F0000A12031C8F2B8A110A128223B8008A1156
:100700000A128F2B03308A003A0882070034013422
:100710000234043408341034203440348034080067
:02400E00753DFE
:00000001FF
